:020000040000FA
:10000000B002001081010000890100008B01000096
:100010008D0100008F010000910100000000000030
:10002000000000000000000000000000930100003C
:1000300095010000000000009701000099010000F8
:100040009B0100009B0100009B0100009B01000040
:100050009B0100009B0100009B0100009B01000030
:100060009B0100009B0100009B0100009B01000020
:100070009B0100009B0100009B0100009B01000010
:100080009B0100009B0100009B0100009B01000000
:100090009B0100009B0100009B0100009B010000F0
:1000A0009B0100009B0100009B0100009B010000E0
:1000B0009B0100009B0100009B0100009B010000D0
:1000C0009B0100009B0100009B01000000F002F872
:1000D00000F047F80AA090E8000C82448344AAF19B
:1000E0000107DA4501D100F03CF8AFF2090EBAE899
:1000F0000F0013F0010F18BFFB1A43F0010318475C
:10010000741E0000941E0000103A24BF78C878C105
:10011000FAD8520724BF30C830C144BF04680C600D
:10012000704700000023002400250026103A28BF55
:1001300078C1FBD8520728BF30C148BF0B60704759
:10014000662900F0D880002070471FB500F0CAF87B
:1001500004000020002101F061FBE0601FBD10B52C
:1001600010BD00F019FF1146FFF7EFFF00F003FB91
:1001700000F037FF03B4FFF7F2FF03BC00F078FF95
:100180000948804709480047FEE7FEE7FEE7FEE72B
:10019000FEE7FEE7FEE7FEE7FEE7FEE70448054967
:1001A000034A054B70470000A9040000CD00000081
:1001B000B0000010B0020010B000001053EA020CB2
:1001C00000F069802DE9F04B4FF00006002B1FBFB7
:1001D000B3FA83F503FA05F424FA05F65E4012BF7C
:1001E0001643B2FA82F502FA05F4C5F120051EBFE6
:1001F00022FA05FC44EA0C04203556EA044C4FEA86
:10020000144418BF641C4FF000084FF000099042DE
:1002100071EB030C39D3002919BFB1FA81F701FA48
:1002200007F6B0FA80F700FA07F6C7F120071EBFFD
:1002300020FA07FC46EA0C062037B6FBF4FCA7EBD5
:100240000507103F07F01F0BCBF120060CFA0BFB44
:100250002CFA06F644BFB3460026202FA4BF5E4604
:100260004FF0000B5BEA060C08BF4FF0010B19EBD7
:100270000B09ABFB027C48EB0608C01B06FB02CC5B
:100280000BFB03CC71EB0C01C1E70B460246414668
:100290004846BDE8F08B13B54FF000004FF0000169
:1002A000AFF30080BDE81C40704700000FB41CB5E0
:1002B000074B06AA7B4469460090059800F061FD53
:1002C0000020694600F009F81CBC5DF814FB000032
:1002D000230000007047704770470A6802F8010B5E
:1002E0000A607047004870476C0000100048704773
:1002F0004C000010704700F005BC0000FFFFFFFF3E
:100300002DE9F04781480068C0F3016003287CD1E3
:100310007F48006810F0030006D0012833D002287F
:100320005FD003282ED100E000BF78480068C0F3FA
:10033000074000F101044FF002017648D0F8880030
:10034000C0F30E0000F10100A1FB0001724B4FF061
:10035000000CA0FB037901FB039100FB0C1122466A
:1003600063463846FFF72AFF05466C480068C0B26E
:1003700000F1010422464FF000032846FFF71EFF5C
:10038000674908605DE061480068C0F3074000F11C
:1003900001044FF002015F48D0F88800C0F30E005E
:1003A00000F10100A1FB00105E4A4FF0000CA1FB20
:1003B000027900FB029001FB0C012246634638469D
:1003C000FFF7FCFE054655480068C0B200F1010485
:1003D00022464FF000032846FFF7F0FE5049086020
:1003E0002FE04A480068C0F3074000F101044FF0D5
:1003F00002014848D0F88800C0F30E0000F1010067
:10040000A1FB00124FF4004000E01BE04FF000039E
:10041000A1FB007902FB009001FB03012246384654
:10042000FFF7CCFE05463D480068C0B200F101046C
:1004300022464FF000032846FFF7C0FE3849086007
:1004400000BF2FE03248006810F0030006D00128FA
:1004500010D0022819D0032823D100E000BF2F4874
:100460000068C0B200F101002B49B1FBF0F02C494B
:10047000086016E029480068C0B200F1010029496F
:10048000B1FBF0F0264908600BE024480068C0B2D8
:1004900000F101004FF40041B1FBF0F02049086089
:1004A00000BF00BFBDE8F08720201F490860194841
:1004B000D0F8A00110F0200F05D000BF1A48006846
:1004C00010F0400FFAD00320144908601748114972
:1004D000C1F8A8011648174908604FF001000C49FF
:1004E00008604FF00400A1F10401086012481349AC
:1004F00008604FF480700749C1F8C80108460068D9
:1005000020F4704040F480400860704788C00F407D
:100510000CC10F4000C00F4000093D0004C10F4056
:1005200000000010001BB700A0C10F4055515155ED
:1005300055545554ACC10F40DEF7EFEFC4C00F4027
:100540004FF4FC51D348C183D3480068D149486176
:10055000D248006818B94FF00060C86106E0CF4883
:100560000068012802D1C006CA4988614FF0805056
:10057000C84988610020CA49086004E0C84800688A
:10058000401CC7490860C64800683228F6DB4FF0B7
:100590008050C049C861704700B5C248007800F07B
:1005A000F000C004BC490860FFF7CAFFBD480078EE
:1005B00000074009B8490860FFF7C2FF0020B849AA
:1005C000086004E0B6480068401CB5490860B448BB
:1005D0000068B0F57A7FF5DB00BD00B5B248B349DD
:1005E0004860C00CAB4948800146AA48C18300203E
:1005F000AA490860AA49086004E0A9480068401CAC
:10060000A7490860A6480068B0F5486FF5DB0020F0
:10061000A749086019E04FF0C0709F490860FFF7D4
:100620008FFF00209E49086004E09D480068401C40
:100630009B4908609A48006847F230518842F4DBD1
:100640009B480068401C9A49086099480068032844
:10065000E1DB4FF0807090490860FFF771FF0020E8
:100660008F49086004E08E480068401C8C4908608F
:100670008B48006847F230518842F4DB28208949D2
:100680000860FFF789FF00208549086004E084487E
:100690000068401C824908608148006847F2305178
:1006A0008842F4DB01207F490860FFF775FF0020D6
:1006B0007B49086004E07A480068401C784908607B
:1006C0007748006842F210718842F4DB06207549D1
:1006D0000860FFF761FF00207149086004E070487E
:1006E0000068401C6E4908606D480068B0F5487F9E
:1006F000F5DB80206B490860FFF74EFF002068495A
:10070000086004E066480068401C65490860644869
:100710000068B0F5487FF5DB0F2062490860FFF7FD
:100720003BFF00205E49086004E05D480068401C13
:100730005B4908605A480068B0F5487FF5DB00BDAA
:1007400000B5024600205A4908600EE0584800688B
:10075000105C54490860012050490860FFF71CFFF5
:1007600053480068401C5249086051480068105CBA
:100770000028EBD100BD4F48006800F410404E49FE
:10078000C1F8C4004FF070404849C8604B484C491C
:100790000860FFF722FF7BE00020404908608020CE
:1007A00040490860FFF7F8FE00204649086004E071
:1007B00044480068401C434908604248006847F2CA
:1007C00030518842F4DB40483D49086000203D49F3
:1007D000086004E03B480068401C3A49086039481A
:1007E0000068B0F5FA6FF5DB00BF3548006A10F01D
:1007F000004F04D13248406A10F0004FF5D0304924
:10080000096AC1F30B1001F00DFB3049086008467E
:10081000006801F0DBFA06462D4A2E4B01F0EEF897
:10082000044601F011F8294908600846006801F003
:10083000CDFA294A03C22249496AC1F30B1001F0DB
:10084000F1FA264908600846006801F0BFFA06463A
:100850001F4A204B01F0D2F8044600F0F5FF1F4973
:1008600008600846006801F0B1FA1D4A03C21C483E
:1008700019490CC803C901F0BFF91A4A03C2194843
:1008800019A10CC81948FFF711FD1848FFF758FFC8
:1008900082E7000000C009200800001010000010CE
:1008A000200000100C000010FF3F00FC00C00240C0
:1008B00024000010C4C00F4000C00F4030002100D1
:1008C000004003401C000010200020011400001014
:1008D0002D431CEBE2364A3F2800001018000010A0
:1008E000380000103000001025665600400000104F
:1008F0002DE9F0410E460446002020622046E168C2
:10090000884730B3252805D0D4E901219047206AD3
:10091000401CF2E7E168204600278847050018D010
:10092000A5F14100192802D820354FF4006732465E
:10093000294620462760FFF703FC40B1012804D078
:10094000F61D26F007060836D8E7361DD6E72846F6
:10095000DAE7206ABDE8F08170472DE9FF4F0C46C9
:100960001E464FF0FF378BB0D2E90001DDF8608002
:100970000A908A46C1F30A5505B93D46002108464A
:100980004FF00000BAF1000F00F4400005DA00EB70
:1009900080004FF4400101EA50004FEA9059B9F14C
:1009A000010F00DDB9460A9850EA4A000ED044F61D
:1009B0001050A5F2FF3545432F14B8F1000F1ED09B
:1009C0007542291E1EDDC9F100021CE0B8F1010FBD
:1009D0004FF0000001D0302103E0F24305E0215444
:1009E000401CB042FBDB30460022002121540B9911
:1009F000C1F80880C1E900200FB0BDE8F08FBD1B31
:100A00006D1CDEE74A4600DA694206A800F052FA99
:100A100006AB07CB03AB07C350460A9900F02EFB89
:100A20008DE80700A0F500501F3800900398002DB6
:100A300009DD42F21F014A46084403A903906846B3
:100A400000F08DFD08E0A0F500504A461F3803A9CC
:100A50000390684600F097FD8DE807000004000C45
:100A600003D04FF0FF30410800E01046B8F1000F0E
:100A700003D00022009215461FE0751E06D400F038
:100A800093F902F1300262556D1EF8D5B34601228A
:100A9000084302D000227F1C04E02078302801D1D6
:100AA00000227F1E002A099787D01DE0112D07DA4A
:100AB00000F07AF9303262556D1C50EA0102F5D12E
:100AC00008430FD10021681E05E0235C625C63547B
:100AD000491C2254401E8142F7DBAB46A81B401E36
:100AE000099001E0009848B1002004F80B000B9831
:100AF000099AC0F80880C0E9002B7DE711264FF065
:100B000000085AE72DE9F04F88460446D21D22F02E
:100B1000070191B0D1E90001CDE90A0100F069FEB9
:100B200002460B98C00F01D02D2007E020688107F6
:100B300001D52B2002E0202101EAC000032A099000
:100B400001D0072A05DB03464146204600F072F932
:100B50000FE12078800601D5E06900E00620B8F1B9
:100B6000650F814606D0B8F1660F18D0B8F1670F4F
:100B700072D132E00020B9F1110F009001DB112396
:100B800001E009F101030AAA01A90CA8FFF7E5FE9B
:100B9000DDE90C70002609F10105834648E00120DB
:100BA0004B4600904FF000470AAA01A90CA8FFF796
:100BB000D4FEDDE90DB00C995D46002618B909F1A7
:100BC000010001EB0005B9EB050003D4C0F1FF36CD
:100BD00009F10105A5EB09002BE0B9F1010F01DADC
:100BE0004FF001090020B9F1110F0090484601DDD6
:100BF000112300E003460AAA01A90CA8FFF7ADFEE5
:100C0000DDE90C704D4600268346207800070AD4A3
:100C1000AB4500DA5D4601A8012D04DD411911F84C
:100C2000011C302907D04F4502DA17F1040F04DA0E
:100C30000120824610E06D1EEEE7002F02DCED1B66
:100C40003E4403E0781CA84200DD0546A7EB060001
:100C500000F1010A4FF000472078000703D4AA45AD
:100C600001DB4FF0FF3A0021B7F1004F0DF14308CF
:100C70008DF8431023D002202B23002F01DA7F426E
:100C80002D234FF00A0C011EA0F1010000DC4FB132
:100C900097FBFCF10CFB11720F4602F1300208F8D1
:100CA000012DF0E7A8F1010003702188090501D5A5
:100CB000452100E06521A0F1010800F8011C099818
:100CC0000FA9A1EB080707F1070700B1012000EB0E
:100CD000050101EBEA70A1693844A1EB0000A0F125
:100CE0000100A0612078C00602D42046AFF3008046
:100CF000099830B1D4E901219047206A00F1010040
:100D000020622078C00620D52046AFF300801CE08A
:100D1000002E04DBB34502DD01A8805D00E0302039
:100D2000D4E901219047206A761C401CBAF1010ADF
:100D300020620AD1FFF7D6FAC0680168405CD4E9A6
:100D400001219047206A401C2062281EA5F1010560
:100D5000DEDC07E0D4E9012118F8010B9047206A96
:100D6000401C2062381EA7F10107F3DC2046AFF3D8
:100D70000080022011B040E601694A1C0261087837
:100D8000704700B58FB0CDE90131002105910549CB
:100D90007944CDE9031011466846FFF7A9FD0FB06D
:100DA00000BD0000E5FFFFFF30B5B0F10A024FEAD9
:100DB000900E71F100034EEA817EB0EB0E0061EB04
:100DC00091014FEA101E4EEA017E10EB0E0041EB3E
:100DD00011114FEA102E4EEA016E10EB0E0041EB9E
:100DE00011214FEA104E4EEA014E10EB0E0041EB7E
:100DF0001141401841F100014FEAD00040EA417032
:100E00004FEAD10110EB80054FEA810444EA907467
:100E100044EB01046D1944EB0404521BA3414FF051
:100E2000000348BF0A3200D530BD401C41F100012B
:100E300030BD00002DE9F0411F460446032601683D
:100E4000072A01F4006004DB08B116A505E016A529
:100E500003E008B115A500E015A521F01000206001
:100E6000A069C01EA0610FB1401EA0612046AFF373
:100E700000804FB1D4E9012138469047206A401CD8
:100E80002062C01C206206E0206AFAE7D4E9012152
:100E900015F8010B9047761EF8D22046AFF300807C
:100EA000BDE8F0814E414E006E616E00494E460035
:100EB000696E66002DE9F047814616468AB03548CE
:100EC0007844D0E9002380680092CDE901303148B0
:100ED00078440C38D0E90223006903924FF03702BE
:100EE000CDE9043041F69B30014491FBF2F0A0F1D2
:100EF000800502FB10141B3C02D56442012000E077
:100F00000020DFF890A080460027FA44AAF1C60A24
:100F10000DE0E00709D03246684607EB47010AEBCF
:100F2000810100F030FB8DE8070064107F1C002C6D
:100F3000EFD1184F7F44B43F17E0E80713D007EB19
:100F400004100DF1180A90E80E00AAE80E00C0681F
:100F5000F04201D198190890324606A903A800F082
:100F600012FB03AB07C36D10641C002DE5D13246A4
:100F70006946B8F1000F03A802D000F0F0FA01E0D2
:100F800000F001FBC9E90001C9F808200AB0BDE87A
:100F9000F0870000981000007546FFF7A7F9AE46ED
:100FA00005006946534620F00700854618B020B575
:100FB000FFF7F4F8BDE820404FF000064FF00007BF
:100FC0004FF000084FF0000B21F00701AC46ACE8F1
:100FD000C009ACE8C009ACE8C009ACE8C0098D465E
:100FE00070470446AFF300802046FFF7C3F80000C7
:100FF0004FF0013C50F8042B51F8043B9A4221D1A8
:10100000A2EB0C03934313EACC1317D150F8042B33
:1010100051F8043B9A4215D1A2EB0C03934313EA17
:10102000CC130BD150F8042B51F8043B9A4209D150
:10103000A2EB0C03934313EACC13DBD04FF0000078
:10104000704700BFD01A01BAB1FA81F101F018015E
:1010500022FA01F0CB40C1F12001DBB2C0B2C01ACC
:101060002CFA01F3D11A914311EAC311E6D170476A
:1010700001491820ABBEFEE7260002005FEA400CE3
:1010800008BF91F0000F4FEA8C234FEAC12243EAD8
:1010900051514FEA1C5018BF00F5F0404FEA3000A4
:1010A00018BF41F000415FEA6C5C00F02980BCF1A0
:1010B000FF3F08BF40F080407047130C06BF12048A
:1010C0004FF0100C4FF0000C130E04BF12020CF185
:1010D000080C130F04BF12010CF1040C930F04BF92
:1010E00092000CF1020CD30F04BF52000CF1010C62
:1010F00011464FF00002A0F11F00A0EB0C0070475A
:1011000011F0004F08BF704731F000413FF4D5AFF8
:101110000B0C06BF09044FF0100C4FF0000C0B0E27
:1011200004BF09020CF1080C0B0F04BF09010CF1FC
:10113000040C8B0F04BF89000CF1020CCB0F04BF11
:1011400049000CF1010CCCF12003A0EB0C0022FAB9
:1011500003F302FA0CF241EA030100F101007047C7
:1011600020F07F4C80EA030023F07F47ACEB0703BD
:1011700003F57C5300F0004003F1FF032DE98049A3
:101180004FEA154B09B44FEA144325EA0B4E24EA03
:1011900003480FF2042606EB132749083E785FEA5E
:1011A000320203FB0667C7F5000707FB06F64FEAA6
:1011B00054374FEAD64606F1020607FB066CCCF11F
:1011C000005C4FEA1C472CEA074C07FB06F40CFBBB
:1011D00006F504EB15464FEA961634BF00204FF093
:1011E00000404FEAD13706FB07FC4FEA1C4C0CFBD2
:1011F0000BF7D21B03FB0CF761EB07010CFB0EF79F
:10120000B0EB074072EB17420CFB08F734BFA2EBC0
:101210000742B2EB074261EB17414FEA0C444FEA39
:10122000910706FB07FC4FEA1C4C0CFB0BF7B0EBDD
:10123000C74072EB573203FB0CF734BFA2EBC74237
:10124000B2EBC74261EB57310CFB0EF7B0EBC700B6
:1012500072EB57720CFB08F734BFA2EBC702B2EB7C
:10126000C70261EB5771039F4FEA816141EA921116
:1012700004EBCC044FEAD1374FEA826206FB07FC4D
:1012800042EA90124FEA80604FEA1C4C0CFB0BF7CD
:10129000D21B03FB0CF761EB07010CFB0EF7B0EB65
:1012A000074072EB17420CFB08F734BFA2EB074272
:1012B000B2EB074261EB17414FEA8C554FEA9107B9
:1012C00004EB9C2406FB07FC4FEA1C4C0CFB0BF7C1
:1012D000B0EBC74072EB573203FB0CF734BFA2EB05
:1012E000C742B2EBC74261EB57310CFB0EF7B0EBD4
:1012F000C70072EB57720CFB08F734BFA2EBC702B2
:10130000B2EBC70261EB577115EB4C254FEA8161D7
:1013100041EA92114FEA82624FEAD13742EA9012D3
:1013200006FB07FC44F100044FEA80604FEA1C4CC6
:101330000CFB0BF7D21B03FB0CF761EB07010CFB5B
:101340000EF7B0EB074072EB17420CFB08F734BF07
:10135000A2EB0742B2EB074261EB174115EB1C15FC
:101360004FEA813141EA92414FEA823242EA9042A9
:101370004FEA80304FEA0C7644F1000448EA034318
:101380004EEA0B484FF0000EB2EB080C71EB03076E
:1013900024BF624639464EEB0E0E4FF0000B00188C
:1013A000524149414BEB0B0BB2EB080C71EB0307BD
:1013B0007BF1000B24BF624639464EEB0E0E4FF018
:1013C000000B0018524149414BEB0B0BB2EB080CE0
:1013D00071EB03077BF1000B24BF624639464EEBED
:1013E0000E0E51EA020718BF46F0010616EB0E7604
:1013F00055F1000254F1000103D5BDE88901BDE8B3
:101400000088BDE88901BDE80048B619524141EBAA
:101410000101A3F10103704780807F7E7D7C7B7A90
:101420007978777676757473727171706F6E6E6D90
:101430006C6C6B6A6A696868676666656464636336
:1014400062616160605F5F5E5E5D5D5C5C5B5B5ABC
:101450005A59595858575756565555555454535329
:1014600052525251515050504F4F4F4E4E4D4D4D84
:101470004C4C4C4B4B4B4A4A4A49494948484847CF
:10148000474747464646454545444444444343430D
:101490004342424242414141002B26D4770021D0B1
:1014A0001CB54FEA370703B44FF010004FF010019E
:1014B0004FF000000FBCBDE810400BF1010BBBF179
:1014C000010F08BF5FEA170722BF12F1010211F1F5
:1014D00001014FF0004143F1000300F0004043EAF6
:1014E00000007047F9D35708DAE746EA064613F1D9
:1014F000400F4FEA16461FDD13F1200FDFBF1643E2
:101500000A46002120335B42C8D0C3F1200746EAD7
:10151000064602FA07F74FEA164646EA0706C3F1FF
:10152000200722FA03F201FA07F721FA03F14FF03C
:10153000000342EA0702B1E746EA020646EA064627
:101540004FEA164646EA0106BCBF46EA0646360C96
:101550004FF000034FF000024FF000019EE72DE92D
:10156000C048934630B491E8380007C831EA400CCF
:1015700048BF34EA430C03D5FFF7F2FDFFF78CFFB9
:10158000F0BCBDE800882DE9C048934630B491E82E
:10159000380007C810F0804F08BF13F0804F03D108
:1015A00000F005F8FFF778FFF0BCBDE8008820F0F8
:1015B0007F4780EA030023F07F4C07EB0C03A3F581
:1015C0007C5300F00040A3F1FE0392F0000F00F006
:1015D000B38095F0000F00F077802DE901494FEAC4
:1015E00011404FEA144621EA004800FB06FC24EAB9
:1015F000064708FB06F607FB08F800FB07F718EBA1
:1016000006484CEB164C4FEA124B18EB07484FEAD2
:1016100015464CEB174022EA0B4E0BFB06FC25EA65
:1016200006470EFB06F607FB0EFE0BFB07F71EEB4D
:10163000064E4CEB164C4FF000061EEB074E4CEBE3
:10164000174B18EB0B0840F1000018EB0E0B58EB92
:10165000000840F100008F1A4FF000013CBFC94361
:10166000661B14BFB5EB040C00213CBFC943F61B3D
:101670004FEA17444EEA8E0E27EA04454FEA1C470C
:1016800004FB07622CEA074C05FB07F70CFB05F689
:1016900004FB0CFC16EB074642EB174216EB0C461C
:1016A00042EB1C421BEB060658EB0202414146EAA4
:1016B0009E0601D5BDE80189B619524141EB0101F1
:1016C000A3F10103BDE801894FEA14454FEA114730
:1016D00024EA054621EA074C05FB07F406FB07F759
:1016E0000CFB06F105FB0CFC11EB074144EB174426
:1016F0004FEA124711EB0C4144EB1C4422EA074C21
:1017000005FB07F206FB07F70CFB06F605FB0CFCD6
:1017100016EB074642EB174216EB0C4642EB1C4514
:101720006A1854F1000148BF7047B619524141EBA5
:101730000101A3F10103704795F0000F37D04FEA84
:1017400011424FEA144721EA024624EA074C02FB01
:1017500007F106FB07F70CFB06F402FB0CFC14EB8D
:10176000074441EB17414FEA154714EB0C4441EB9A
:101770001C4125EA074C02FB07F506FB07F70CFBAB
:1017800006F602FB0CFC16EB074645EB174516EB7D
:101790000C4645EB1C42121951F1000148BF70473D
:1017A000B619524141EB0101A3F1010370474FEA21
:1017B00014454FEA114724EA054621EA074C05FB88
:1017C00007F106FB07F70CFB06F24FF0000605FBDE
:1017D0000CFC12EB074241EB174112EB0C4251EBB0
:1017E0001C4148BF7047921841EB0101A3F101036E
:1017F0007047490050EAC12018BF04204A0D18BFA5
:1018000040F0010040F2FF72B2EB515F08BF40F0C0
:101810000200012808BF05207047000010B500290C
:101820000AD00878002807D005487844FFF7E0FB85
:10183000002801D0002010BD0248784410BD0000EF
:101840006A0700006207000021F00042A2F1605226
:10185000B2F5801F01F0004328BFD2F17F6C0BD995
:101860005FEA001C43EAC20242EB507018BF7047A7
:1018700028BF20F001007047B2F5801FBCBF18469A
:1018800070474FEA410C1CF5001F02D2084600F0D9
:1018900022BB70B500F05CF900000089FFF7F6BFCD
:1018A0004FF00040A0F580007047000010B591EAAD
:1018B000030F48BF83F0004300F1A681841A71EB47
:1018C000030C05D2121943EB0C03001B61EB0C0156
:1018D000DFF824E14FEA1154A4EB135C1EEA430F36
:1018E00018BF9EEA445F73D023EA0E03DCF1200E9A
:1018F00021EA045143F4801332D322FA0CFE10EB98
:101900000E0023FA0CFE41EB0E01CCF1200E03FA7F
:101910000EFE10EB0E0051F10001B1F5801FCCF16D
:10192000200E32D201EB045112FA0EF2BDE8104043
:1019300058BF7047401C38BF5FEA420218BF70476B
:10194000002814BF20F0010041F100014FEA4103DB
:1019500013F5001F38BF7047A1F1C04100F046B930
:10196000012A43EB0302ACF1200CDCF11F0E32BF65
:101970004FF0000E23FA0CF310EB030041EB04517F
:10198000B4EB115FD0D0A1EB045101F580114908EF
:101990005FEA300001EB04510ED350F1000038BF74
:1019A00012FA0EFE08D1BDE81040C9E7401C38BF4E
:1019B0005FEA4202CAD1C3E7BDE810404FEA4103E3
:1019C00013F5001F38BF7047A1F1C04100F00EB9F8
:1019D0009EEA445F08D011EA5E0FBDE8104004BFE4
:1019E00001F0004100207047BDE8104070B500F0E4
:1019F000AFF800BF64FBBE3E0000E0FFDFF848C167
:101A000070B51CEA111E1EBF1CEA13159EEA0C0FCE
:101A100095EA0C0F00F06F8081EA030423EA4C136F
:101A20004EEAD47E21EA4C1141F4801143F4801334
:101A3000AE44A1FB024CA0FB0365AEF17F7E3619DC
:101A400055EB0C05A1FB034C4CF10003A0FB021C61
:101A500016EB0C06654153F10003094218BF46F02E
:101A6000010613F4007F0BD14FEA03314FEA053032
:101A7000340341EA155140EA16506FF003020AE0C0
:101A80004FEAC3214FEAC520F40241EA555140EA2A
:101A900056506FF0020202EB2E4201EB025585EA2E
:101AA000CE710AD05FEA440C18BF24F0004450F114
:101AB000000041F1000120EAD47040F2FE7C624552
:101AC00000D270BDA84214BF4FF080444FF0404494
:101AD000002E08BF0024BEF1806FA8BFA1F1C04155
:101AE000BDE8704080F282804FF0000001F1C041FB
:101AF00001F0004170479EEA0C0F0CEA131518BF65
:101B000095EA0C0F06D04FF0000081EA030E0EF0AC
:101B1000004170BD00F01CF88900013E00F007B8DC
:101B200000F009B84FEA430C5FEA5C5C08D081EA38
:101B3000030100F05BB84FEA410C5FEA5C5CF6D150
:101B40004FF00000014970470000FF070000F87FD8
:101B50000EF1020E2EF0030E5EF8046B364205D431
:101B6000012A43EB030515F5001F12D8012841EBAC
:101B7000010C1CF5001F0CD80ED14FEAD17C15F5D5
:101B8000001F0CEB4C0C0CF1020C08BF4CEBD37C8F
:101B900004E04FF0080C01E04FEAD37C0CEB4C055D
:101BA00026FA05F606F00706B6F1040C06D20EEB8F
:101BB000860CBDE870404CF0010C6047DFE80CF08B
:101BC000090B02024FF000414FF00000A1F5002187
:101BD00070BD19461046012851EB010418BFD4F519
:101BE000001484BF002001F0004170BD0808A0F57A
:101BF00000114FEA3101704710B591EA030F48BF59
:101C000083F000433FF55AAE841A71EB030C07D200
:101C100012198CF0004C43EB0C03001B61EB0C0120
:101C2000DFF8A4E14FEA1154A4EB135C1EEA430F62
:101C300018BF9EEA445F00F0B08023EA6E03524270
:101C400021EA0451C3EB6E0338BF5B1EDCF1200EAA
:101C500025D322FA0CFE10EB0E0043FA0CFE41EBEA
:101C60000E01CCF1200E03FA0EFE10EB0E0051F126
:101C70000001CCF1200E29D412FA0EF201EB04512E
:101C8000BDE8104058BF7047401C1CBFB2F1004F68
:101C9000704700280CBF491C20F00100704712EB70
:101CA000020E43EB030218BF4FF0010E4EEA420250
:101CB000ACF1200CDCF11E0E54D943FA0CFE10EBF3
:101CC0000E0051F1FF31CCF11E0ED5D50EF1010EF3
:101CD00012FA0EFE404141EB010101EB445C5FEA68
:101CE0005C5C10D910EBDE7001EB045138BFBEF123
:101CF000004FBDE8104018BF704700280CBF491CBA
:101D000020F00100704730D24FEAD42C11F50011B9
:101D100024F400641BD0B1FA81F20B3AA41AA41E79
:101D2000D2F12003914030FA03F31943904001EBC4
:101D3000CC71002C01EB0451BDE81040A8BF7047E6
:101D400001F1C0414FF0000001F000417047B0FACE
:101D500080F310FA03F100D110BDE41A173C4805D6
:101D6000C90AE4E701EB045110BD491001EB04512D
:101D7000BDE810404FEA300002E04FF0000170472C
:101D80004A0008BF0042F8D0B2F5001F28BF7047D4
:101D900001F000414FF0000070479EEA445F07D019
:101DA00011EA5E0FBDE8104004BF0021002070471B
:101DB000BDE8104070B5FFF7CBFE00BF40DFF63E38
:101DC00083F00041104670470000E0FF43004FEAF7
:101DD000D30C4FEA3C0C43401FBF40070CF160514D
:101DE00013F0FE4F70471CF0006F03D100200CF081
:101DF000004170470CF0004343EA507010B540EAD0
:101E0000CC0000F022F800BF000000924FEA000171
:101E1000FFF7ECBE4FF000414FF00000A1F50021AC
:101E200070470000B0FA80F310FA03F2C3F19D038B
:101E30000AD0D90501EB1220530638BF704700F1D4
:101E4000010008BF20F0010070470EF1020E2EF0D5
:101E5000030E5EF8044B244204D44FEA4102B2F16F
:101E60007F4F11D84FEA4003B3F17F4F0CD80ED10A
:101E70004FEAD07CB2F17F4F0CEB4C0C0CF1020C12
:101E800008BF4CEBD17C04E04FF0080C01E04FEAB6
:101E9000D17C0CEB4C0324FA03F404F00704B4F1F6
:101EA000040C06D20EEB840CBDE810404CF0010C83
:101EB0006047DFE80CF0070802024FF00040A0F591
:101EC000800010BD0846420018BFD2F1807288BF62
:101ED00000F0004010BDFF2141EAD050C00570471E
:101EE00002400000000000A00000000005400000CB
:101EF000000000C8000000000C4000000000409CF2
:101F000000000000194000000020BCBE00000000DE
:101F100034400000BFC91B8E00000004B540000023
:101F2000504BCFD06607E2CF010000006C410000AB
:101F30003E8251AADFEEA73401000000D942000022
:101F4000DCB5A0E23A301F97FFFFFFFFB445000069
:101F5000FD25A0C8E9A3C14FFFFFFFFFFF3F000021
:101F60000000008000000000FF3F00000000008033
:101F700000000000B01F0000000000104000000042
:101F800008010000F01F0000400000107002000077
:101F9000240100001C00000043000000F8FFFFFFC8
:101FA0000C0000000E0000000F0000002E000000DA
:101FB000C0C62D000000000000000000000000006E
:101FC0000000000000000000000000000000000011
:101FD0000000000000000000000000000000000001
:101FE00000000000000000000000000000000000F1
:040000050000018175
:00000001FF
